:100000000C945E010C947B010C9496010C947B0182
:100010000C947B010C947B010C947B010C947B0170
:100020000C947B010C947B010C94DA190C947B01E9
:100030000C947B010C947B010C947B010C947B0150
:100040000C947B010C947B010C947B010C947B0140
:100050000C947B018E058E05BA05BA051C063A067E
:10006000520752074506DE06EF06EF062900140088
:100070001A000800150017001C0018000C001200E0
:1000800013002F00300031002B0004001600070081
:1000900009000A000B000D000E000F0033003400B1
:1000A0002800A800E1001D001B0006001900050043
:1000B000110010003600370038000000E500015143
:1000C000E000E300E20000002C000000015100000D
:1000D0002A0000000000E600E700E4000000000045
:1000E0000000000000000000000000000000000010
:1000F000000000000000000035001E001F0020006E
:1001000021002200230024002500260027002D00C6
:100110002E00010001003A003B003C003D003E0083
:100120003F00400041004200430001000100010087
:100130000100440045000100010001000100010030
:1001400001000100010000000100010001000100A8
:10015000010000000100000001000000010000009B
:10016000000001000100010000000000000000008C
:10017000000000000000000000000000000000007F
:100180000000000009023B00020100A0FA0904007F
:1001900000010301010009210101000122400007C3
:1001A00005810308000109040100010300000009A2
:1001B0002101010001227B000705830308000112D1
:1001C000011001000000086BB1EEC4120001020032
:1001D000011003430068006500760072006F006E36
:1001E0000000001803520061006D006F006E0020D7
:1001F0000049006D00620061006F00000004030907
:100200000405010902A10185020901A100050919DE
:1002100001290815002501950875018102050109CC
:100220003009311581257F95027508810609381539
:1002300081257F950175088106050C0A3802158114
:10024000257F950175088106C0C005010980A101BF
:10025000850319012AB700150126B700950175100D
:100260008100C0050C0901A101850419012AA00221
:10027000150126A002950175108100C0050109062F
:10028000A101050719E029E7150025019508750169
:1002900081029501750881030507190029FF1500E2
:1002A00026FF0095067508810005081901290595A6
:1002B0000575019102950175039103C011241FBEBC
:1002C000CFE5D8E0DEBFCDBF11E0A0E6B0E0EAE2C6
:1002D000FBE302C005900D92A030B107D9F722E0F0
:1002E000A0E0B1E001C01D92AB3BB207E1F70E9474
:1002F0009E130C94931D0C940000A82FB92F80E03E
:1003000090E041E050EA609530E009C02D918227ED
:100310009795879510F084279527305EC8F36F5F17
:10032000A8F30895EADF8D939D930895CF93CFB7F7
:10033000CF93DF93C395839BE9F7839B10C0839B87
:100340000EC0839B0CC0839B0AC0839B08C0839B09
:1003500006C0C0919202C395C09392028EC06F9363
:10036000C0919102DD27C756DD4F2F9365E5839B32
:1003700003C02F916F91E1CF0F931F934F9320E014
:1003800040E15F9300B30C7003FB27F93F9350E00B
:100390003BE039C01C7040642F77012F5F5F1EC0A7
:1003A000406810B31C702F7752501FC0406400B3D8
:1003B0002F770C70D1F15F5F00C023C0406210B393
:1003C0002F771C7091F15F5F00C025C00C70102763
:1003D000515012F45D5F0000115027952C3F10B36F
:1003E000C8F61C700127015027952C3FC8F64227FC
:1003F000499300B30C7010274F73115027952C3F71
:10040000A8F64695469510B31C7079F00127015067
:1004100027952C3F98F66B5A60F3315000B3B0F635
:1004200000C010E81ABF00271CC03B503195C31B09
:10043000D04010E81ABF0881033C21F10B3411F1C0
:1004400020918E021981110F1213EDCF4A81441FA2
:10045000093679F10D3211F0013E29F74F7009F09C
:10046000042F009397023F915F914F911F910F913D
:100470002F916F91CAB7C7FD5DCFDF91CF91CFBFED
:10048000CF91189520919702222369F3109195023C
:10049000112309F049C034300AF448C03093950262
:1004A00020939002109191023BE0311B3093910216
:1004B0003DC0009195020130BCF50AE54F7049F44A
:1004C0003091790034FD33C000937900CBE6D2E05F
:1004D00032C0433059F0443091F03091760234FD0F
:1004E00026C000937602C7E7D2E025C03091AF0264
:1004F00034FD1DC00093AF02C0EBD2E01CC03091B0
:10050000820234FD14C000938202C3E8D2E013C01B
:10051000052710E000C0000002BB1AC0052710E04C
:10052000221F1DC010E021C04AE502C032ED432F5A
:10053000C4E1D0E032E011B31C60939A02B311BB66
:100540005CE020E865E320FF052702BB27951795AF
:100550001C3FF0F66695B8F7B1F720FF052702BB00
:10056000279517951C3FD0F62795179517FF052758
:1005700000001C3F02BBB0F629913A9519F7037FA2
:1005800010919602110FC651D04002BB11F010938A
:100590008E0210E81ABF086011B3137F402F437F0B
:1005A00054E05A95F1F702BB11BB42BB5CCF662306
:1005B00011F089EA01C08AEA0E943C0581E00895B1
:1005C00081E0089581E008950C94E20208950C946E
:1005D000E6021F93CF93DF9300D000D01F92CDB7D8
:1005E000DEB749835A836B833091030189819A81F5
:1005F000311114C0662359F0222349F00E948F095B
:10060000182F682F89819A810E94380903C00E949F
:100610006309182F69817A81812F04C00E948F0994
:1006200069817A810F900F900F900F900F90DF915A
:10063000CF911F910C940F11FC01262F4081518105
:100640006281738184810C94E90281E00895CF93E3
:10065000DF93EC0160E00E941C03BE01DF91CF91AB
:100660000C94E7020C9455120C94511208950E94B8
:10067000E2070E9436032FEF84E39CE02150804084
:100680009040E1F700C000000C94001A0F931F93F4
:10069000CF93DF938C0161E00E941C03EC01B80151
:1006A0000E94E4028823F1F1B801CE010E9487186C
:1006B0008823C1F1B801CE010E943416882391F13C
:1006C000B801CE010E94E317882361F1F80182810D
:1006D000882309F1CB358DE5D807C1F050F4C11559
:1006E000FCE5DF0781F0CF3DDC45A9F40E94F60E62
:1006F00019C0CC35EDE5DE0761F0CD35DD4559F4A7
:100700000E94390E08C00E9437030CC00E94420E9E
:1007100002C00E94450EC801DF91CF911F910F9139
:100720000C94E00280E0DF91CF911F910F9108952A
:100730000E9484190C94B1030E94B4030C948A198A
:1007400008950C94A00381E008950C94A3030895E8
:10075000CF93C82F0E94A1038C2F0E94A503CF9195
:10076000089580E00C94A8030E94E3180C94A80359
:100770000E94E31890910201891721F080930201F1
:100780000C94A8030895CF93DF93CDB7DEB72B97D2
:100790000FB6F894DEBF0FBECDBF4F835887698771
:1007A0007A878B8761110E94850D9E012F5F3F4FD5
:1007B00086E0F90111928A95E9F785E0FE01379606
:1007C000D90101900D928A95E1F789819A814C8136
:1007D0005D81452B31F09F3F31F491E08F3F19F45B
:1007E00003C091E001C090E090FF09C049815A81A7
:1007F0006B817C818D819E810E94A60C05C0C90100
:100800000E9425038111F2CF2B960FB6F894DEBF1C
:100810000FBECDBFDF91CF910895FC018081918102
:100820000E94D1090895CF93882309F4A4C0C82F4A
:100830008238C1F40E94E31881FD9DC069E3809174
:100840006200909163000E9476190E94A70D2FEF1D
:1008500081EE94E0215080409040E1F700C000001C
:1008600069E319C0833801F50E94E31880FD83C055
:1008700063E580916200909163000E9476190E9466
:10088000A70D2FEF81EE94E0215080409040E1F7DA
:1008900000C0000063E580916200909163000E94B7
:1008A0007819CF910C94A70D8438C1F40E94E318F5
:1008B00082FD61C067E480916200909163000E94B4
:1008C00076190E94A70D2FEF81EE94E02150804011
:1008D0009040E1F700C0000067E4DDCF8CEF8C0FA3
:1008E000813AD0F46C2F80916200909163000E9455
:1008F0004019882349F06C2F809162009091630029
:100900000E9478190E94A70D6C2F8091620090912F
:1009100063000E947619C5CF80E28C0F883048F4BE
:10092000C77081E001C0880FCA95EAF70E94680D80
:10093000B8CFEBE5EC0FE33040F4F0E0E855FF4FC3
:10094000808190E0CF910C940819E8E5EC0FE73135
:1009500050F4F0E0EE0FFF1FE658FF4F80819181C9
:10096000CF910C941E19CD3E30F08C2F0E94231491
:10097000CF910C94F514CF910895882309F464C0A5
:10098000823879F40E94E31881FF5EC069E38091A8
:100990006200909163000E9476190E94A70D69E39E
:1009A00010C08338B1F40E94E31880FF4DC063E5A6
:1009B00080916200909163000E9476190E94A70DB9
:1009C00063E580916200909163000E9478190C9415
:1009D000A70D843879F40E94E31882FF35C067E4DC
:1009E00080916200909163000E9476190E94A70D89
:1009F00067E4E7CF9CEF980F913A10F4682FE1CFAE
:100A000090E2980F983050F4877091E001C0990FF0
:100A10008A95EAF7892F0E946E0DD9CF9BE5980F32
:100A2000933020F480E090E00C94081998E5980F3A
:100A3000973120F480E090E00C941E198D3E20F058
:100A40000E947E140C94F51408951F93CF93DF93A6
:100A5000182FEB010E941304209741F08FE99FE0CB
:100A60000197F1F700C000002197F6CF812FDF91A9
:100A7000CF911F910C94BD04893319F060E070E0B0
:100A800002C060E570E00C942505882321F00E94E7
:100A9000680D0C94A70D0895882321F00E946E0D17
:100AA0000C94A70D0895CF92DF92EF92FF920F93CF
:100AB0001F93CF93DF937C01D62FC72FFC011281A8
:100AC000058102950F700E945E0D8823B9F01123F5
:100AD000A9F08C2F807F803421F080E28D0F883048
:100AE00068F08091520282FD09C082E00E94070EE8
:100AF0000E945E0D91E0D82ED92601C0D12CCC2EBB
:100B0000C2948FE0C8228C2D90E08C30910508F0C3
:100B1000C9C1FC01E65DFF4F0C942B1D8C2F807F1B
:100B2000CF70882311F0C295C07F112399F0CC2398
:100B300009F4A4C180E28D0F883010F0D11104C0F7
:100B40008C2F0E94680D03C08C2F0E94780D0E948C
:100B5000A70D94C18D2F0E94BD04CC2309F4A2C11E
:100B600080E28D0F883038F1DD2329F18C2F0E942F
:100B70007E0D24C08C2F807FCF70803211F0C29503
:100B8000C07FDD2319F0D130A1F140C08091520225
:100B900082FF17C0112349F0CC2329F08C2F0E942B
:100BA000680D0E94A70D80E06AC180E00E94BD042C
:100BB000CC2309F477C18C2F0E946E0D0E94A70DE3
:100BC00071C1112371F0002341F0013031F40E9412
:100BD000880D8C2B0E94900D65C10E94880D8C2B76
:100BE0000EC0002319F0013009F45CC10E949D0D74
:100BF0001FC0112339F0063008F054C18C2F0E9419
:100C0000450550C1053008F04DC112C0112319F03F
:100C10000023A1F333C1002359F0D93309F03FC1B8
:100C2000FFEF07EE13E0F15000401040E1F735C14F
:100C30008C2F0E944C0536C18C2F8695869583702B
:100C400019F0813061F02EC1112321F08D2F9C2FDE
:100C5000937002C080E090E00E9408192BC111231C
:100C600021F08D2F9C2F937002C080E090E00E94B5
:100C70001E1920C18D2F112319F00E94231402C0C8
:100C80000E947E140E94F51415C18C2F837009F008
:100C900047C011110BC12D2F229526952770220FC9
:100CA000220F6D2F6F70862F90E0A0E0B0E0022E33
:100CB00004C0880F991FAA1FBB1F0A94D2F7D4FF44
:100CC00010C04FE050E060E070E004C0440F551FDA
:100CD000661F771F2A95D2F74095509560957095BD
:100CE00003C040E050E0BA01C695C695C3708A01C2
:100CF0009B01082B192B2A2B3B2BC901B801C230B1
:100D000049F058F4C13019F00E944E08CFC00E943B
:100D10003C08CCC00E946008C9C00E943A08C6C006
:100D2000112319F08C2F817001C08695882309F456
:100D3000BDC02D2F229526952770220F220F6D2FD3
:100D40006F70862F90E0A0E0B0E0022E04C0880F04
:100D5000991FAA1FBB1F0A94D2F7D4FF10C04FE0FF
:100D600050E060E070E004C0440F551F661F771F1D
:100D70002A95D2F7409550956095709503C040E054
:100D800050E0BA01C695C695C3708A019B01082B35
:100D9000192B2A2B3B2BC901B801C23049F058F45A
:100DA000C13019F00E94130981C00E9401097EC060
:100DB0000E9425097BC00E94740878C0CF7011235F
:100DC00039F08C2F0E949A088D2F0E9445056EC025
:100DD0008D2F0E944C058C2F0E94BB0867C0D23F0C
:100DE00021F128F4D03F41F0D13FC1F043C0D33FBF
:100DF00019F1D43F79F03EC0112341F0053008F0DD
:100E000051C08C2F8F710E94E0084CC0063008F052
:100E100049C0F7CF8091520282FF18C0112339F0E8
:100E20008C2F8F710E949A083DC01123C9F38C2F1B
:100E30008F710E94BB0836C0112329F08C2F8F714F
:100E40000E9485082FC00E9480082CC0112349F001
:100E5000CF718C2F0E949A0863E08C2F0E94EC0DBA
:100E600021C081E00E94070E0230E0F082E00E9483
:100E7000070E18C0112331F0002391F28D2F0E942C
:100E8000130410C0002399F2D93349F41FEF27EE61
:100E900033E0115020403040E1F700C000008D2FBA
:100EA0000E94BD0488EF8C0D843020F40E94E3186A
:100EB0000E94A803DD20C9F00E945A0D80FD15C0D4
:100EC000F70112820E94540D0E949A08C7010E94E5
:100ED00096070E94540DDF91CF911F910F91FF90C3
:100EE000EF90DF90CF900C94BB08DF91CF911F91D2
:100EF0000F91FF90EF90DF90CF9008950F931F9385
:100F0000CF93DF93EC01688179818A810E94DC09AB
:100F10008C010E9437090E942808B801CE010E9466
:100F20005305DF91CF911F910F910895CF93DF93D8
:100F3000EC01988189812B813C81232B31F08F3FFB
:100F400031F481E09F3F19F403C081E001C080E0EB
:100F500080FD1DC0CE010E944603811110C00E9479
:100F60005E0D8823A1F08A81882389F08091520246
:100F700082FD0DC082E0DF91CF910C94070ECE016F
:100F80000E947E07CE01DF91CF910C942703DF9161
:100F9000CF91089580E090E00E94081980E090E0F1
:100FA0000E941E190E94850D0E94A70D0E94261600
:100FB0000C94F51480916200909163000E947A195C
:100FC0000C94CA070E94750D0C94DA0792959F70D5
:100FD000963079F010F4925001C09A50923068F433
:100FE000803F69F018F4883E40F409C0843F29F43A
:100FF00006C0883E20F0813F11F080E0089581E036
:101000000895FC01808191810E94D1090E94E60728
:101010000895CF93DF9300D000D01F92CDB7DEB7F5
:101020000F900F900F900F900F90DF91CF91089538
:10103000CF93DF9300D000D000D0CDB7DEB7269697
:101040000FB6F894DEBF0FBECDBFDF91CF910895EC
:10105000089508950C9429080C942A080E942C08DD
:101060006093350170933601809337019093380176
:101070000C94CA070C942E080F931F93009135010E
:10108000109136012091370130913801602B712B7E
:10109000822B932B1F910F910C942E080F931F936B
:1010A00000913501109136012091370130913801BE
:1010B00060237123822393231F910F910C942E0898
:1010C0000F931F9300913501109136012091370144
:1010D0003091380160277127822793271F910F9144
:1010E0000C942E080C9429080E9472086093310118
:1010F0007093320180933301909334010C94CA07AA
:1011000060E070E0CB010C9474080F931F9341E0F2
:1011100050E060E070E08A019B0104C0000F111FE5
:10112000221F331F8A95D2F7C901B8011F910F9171
:101130000C9474080F931F9341E050E060E070E05E
:1011400004C0440F551F661F771F8A95D2F7809100
:10115000310190913201A0913301B09134018A01A3
:101160009B01082B192B2A2B3B2BC901B8011F917E
:101170000F910C9474080F931F9341E050E060E0CE
:1011800070E004C0440F551F661F771F8A95D2F781
:101190004095509560957095809131019091320104
:1011A000A0913301B09134018A019B0108231923D6
:1011B0002A233B23C901B8011F910F910C94740895
:1011C0000F931F9341E050E060E070E004C0440FD3
:1011D000551F661F771F8A95D2F780913101909134
:1011E0003201A0913301B09134018A019B0108279B
:1011F00019272A273B27C901B8011F910F910C9489
:1012000074080F931F9300913101109132012091C6
:10121000330130913401602B712B822B932B1F9162
:101220000F910C9474080F931F930091310110914A
:1012300032012091330130913401602371238223E4
:1012400093231F910F910C9474080F931F93009197
:101250003101109132012091330130913401602726
:101260007127822793271F910F910C94740808957A
:101270002EE0929F800D1124E82FE695E695E695E5
:10128000877051E001C0550F8A95EAF785E0E89F25
:10129000F0011124EC5FFE4F20E030E070E040816F
:1012A000CB01022E02C0969587950A94E2F78170D1
:1012B000819584278523842781932F5F3F4F253095
:1012C000310569F708952EE0929F800D1124682F53
:1012D000669566956695982F977085E0689FB00132
:1012E000112440E050E080E0FB01E40FF51FEC5FCB
:1012F000FE4F208130E0092E02C0369527950A94D2
:10130000E2F721703327042E01C0220F0A94EAF776
:10131000822B4F5F5F4F4530510531F70895BF92E3
:10132000CF92DF92EF92FF920F931F93CF93DF93B1
:101330008C01C0903101D0903201E0903301F090E7
:1013400034018091350190913601A0913701B0911F
:101350003801C82AD92AEA2AFB2ACFE1D0E0D701EE
:10136000C6010C2E04C0B695A795979587950A944B
:10137000D2F780FD04C0219790F7B12C07C0BC2E96
:10138000B8018C2F0E9422110197A9F38B2DDF91B8
:10139000CF911F910F91FF90EF90DF90CF90BF9072
:1013A0000895CF93DF93EC010E948F09BE010E9444
:1013B0002211DF91CF9108951F93CF93DF93EB011B
:1013C00090910301992321F0CB010E94D10913C010
:1013D000882349F0CB010E948F09182F682FCE0176
:1013E0000E94380904C0CB010E946309182FBE0176
:1013F000812F0E942211DF91CF911F9108951F9399
:10140000CF93DF93C091390116E080913A01C8175C
:1014100099F0D0E01C9FF0011D9FF00D1124E55CB8
:10142000FE4F4081518162817381848195810E9448
:1014300018082196C770E9CFDF91CF911F910895C9
:1014400040916B0150916C0160916D0170916E0142
:1014500080916F01909170010C94180820913901CE
:1014600090913A0156E02917A9F030E0529FF0011F
:10147000539FF00D1124E55CFE4F7181761306C079
:101480007081781303C07281741306C02F5F3F4FC1
:101490002770E9CF80E0089581E00895EF92FF92F0
:1014A0000F931F93CF93DF938091700182958F707C
:1014B00009F065C080916D01882309F460C08091B6
:1014C0003901F0903A0110916B0100916C0160912B
:1014D0006E0170916F0191E01F3F09F090E0C091A3
:1014E0006000D0916100292F96E0E92E8F1509F454
:1014F00046C06115710521F00F3F21F030E003C0B7
:1015000031E001C0322F90E030FD36C0E89EF0019E
:10151000E99EF00D1124DF01A55CBE4F11963C91B0
:101520001197301329C03C91311326C012963C917B
:101530001297311121C013964D915C911497461B5F
:10154000570B4C175D07C0F4809170018F7080615C
:1015500080937001E05CFE4F80818F70806180839A
:101560008BE691E00E949607DF91CF911F910F913A
:10157000FF90EF900C94FF0901968770B7CFDF9131
:10158000CF911F910F91FF90EF9008958F929F92AE
:10159000AF92BF92CF92DF92EF92FF920F931F9381
:1015A000CF93DF93CDB7DEB761970FB6F894DEBF68
:1015B0000FBECDBF8C0185E0F801DE011D960190C4
:1015C0000D928A95E1F7D8011296EC9090916B01FB
:1015D00020916C0140916E0150916F0141155105B0
:1015E00031F02F3F31F481E09F3F19F403C081E0D7
:1015F00001C080E080FD7CC1F801C080D180838083
:1016000094808BE6A82E81E0B82EF0906D01B40195
:10161000641B750B4091600050916100FF2009F43C
:1016200011C180917001382F307F6417750708F061
:10163000CBC031118AC0D21214C0C91212C0FE2C04
:10164000E1100FC08F708061809370010E94200AAA
:10165000C5010E94960780917001D80115968C9360
:1016600061C18114910439F0BFEFDB1206C081E043
:10167000CB1203C003C081E001C080E080FD03C045
:1016800081E08E2502C080E090E080FF10C04E2DEA
:101690006D2D8C2D0E942E0A882349F08BE691E057
:1016A0000E949607EBE6F1E086E0DF019DC0892805
:1016B00039F0BFEFDB1206C081E0CB1203C003C0DC
:1016C00081E001C080E080FD03C081E08E2502C082
:1016D00080E090E0E82FE170BE2E80FF2CC04E2D00
:1016E0006D2D8C2D0E942E0AF82E811124C0CD86DE
:1016F000DE868D859E850E94D109292F22952F7027
:10170000223018F0243090F405C09F7059F08111F8
:1017100009C008C19F7031F0D80115969C91907F47
:1017200009F400C1805E883008F4FCC0C8010E9442
:101730009607FB2CF7C0FE2CEE2009F4F3C0809135
:10174000700181608093700154C0D21206C0C9122A
:1017500004C0E11002C0F80199C0C8010E9401084C
:10176000882361F1EE2051F120917001822F829542
:101770008F7090E0029774F080916B0190916C01F2
:1017800098878F8319869B868A862C87CE01079639
:101790000E94960786E0F801ABE6B1E001900D9259
:1017A0008A95E1F70E944E0A0E94200A0AC0D216CA
:1017B00011F1C8010E94010881112CC0C8010E94CA
:1017C0009607FF24F394AEC03111F1CF782D998A9A
:1017D000888AA6016E2D89890E9409088BE691E00E
:1017E0000E94960786E0D5011D928A95E9F70E942E
:1017F000200AF12C97C0C912DCCFE110DACFF80132
:101800008583C8010E94960786E0D5011D928A95BE
:10181000E9F788C0EE2091F220917001822F829525
:101820008F7090E002970CF4B5CF80916B0190918E
:101830006C019A8389831B829D828C822E83CE01C8
:101840000196A6CF6417750708F044C0FE2CEE2061
:1018500009F4B4CFD21230C0C9122EC02091700149
:1018600020FD21C0822F82958F70482F50E04115B6
:101870005105C9F0F80125834F30510541F08F5FC4
:10188000982F9295907F822F8F70892B8583C80126
:101890000E94960786E0F801ABE6B1E001900D9258
:1018A0008A95E1F73DC086E0F801ABE6B1E0019032
:1018B0000D928A95E1F736C0C8010E940108811196
:1018C00069CF80917001816080937001C8010E948E
:1018D000960728C0782D998A888AA6016E2D898955
:1018E0000E94090886E0D5011D928A95E9F718C083
:1018F000EE2009F463CFC8010E940108F82E882366
:1019000009F45CCF86E0F801ABE6B1E001900D92FE
:101910008A95E1F78BE691E00E940D040E944E0A41
:101920000E94200A8F2D61960FB6F894DEBF0FBE7D
:10193000CDBFDF91CF911F910F91FF90EF90DF907E
:10194000CF90BF90AF909F908F9008951F93CF93AB
:10195000DF93CDB7DEB72C970FB6F894DEBF0FBE7E
:10196000CDBF4F83588769877A878B879C87CE0145
:1019700007960E94C60A8823D1F09F8188852A8510
:101980003B85232B31F08F3F31F481E09F3F19F4E9
:1019900003C081E001C080E080FD47C04F815885D1
:1019A00069857A858B859C850E9418083EC086E0F3
:1019B000FE013796DE01119601900D928A95E1F7AE
:1019C000FF81E8856A857B856115710531F0EF3F00
:1019D00031F481E0FF3F19F403C081E001C080E0F1
:1019E00080FD23C020913A0130E0C9010196877043
:1019F00099274091390150E084179507F1F1F98357
:101A0000EA837D836C8396E0929FD001939FB00D13
:101A10001124A55CBE4FFE01319601900D929A955E
:101A2000E1F780933A010E94FF0916E080913901A5
:101A300090913A01891771F1189FC0011124855CBA
:101A40009E4F0E94C60A882329F1E09139011E9F0A
:101A5000F0011124E55CFE4F408151816281738168
:101A6000848195810E9418088091390190E0019647
:101A70008770992780933901D9CF0E94E20710928D
:101A80003A0110923901EBE6F1E086E0DF011D92A8
:101A90008A95E9F72C960FB6F894DEBF0FBECDBF3E
:101AA000DF91CF911F91089580917901859585955A
:101AB00085950895809179018770089590917901B5
:101AC000977081E009F480E0089580918401089581
:101AD00090918401892B8093840108958095909141
:101AE00084018923809384010895109284010895CC
:101AF00090918301892B8093830108958095909123
:101B000083018923809383010895109283010895AE
:101B100080917A01089508950C948B0D0C948C0D8E
:101B20009091520292FD08C090917A01981721F08D
:101B300080937A010C948E0D089580917A01882308
:101B400029F010927A0180E00C948E0D0895CF93C5
:101B5000DF93E0916200F0916300809184018083C3
:101B6000E0916200F0916300908180918301892B64
:101B7000808380917A01882381F0E0916200F09166
:101B800063009081892B8083809162009091630033
:101B90000E94341981110E949D0DC0916200D09164
:101BA000630048E050E061E771E0CE010E94451D0E
:101BB000892B69F088E0FE01A1E7B1E001900D9268
:101BC0008A95E1F7CE01DF91CF910C94EF18DF9168
:101BD000CF9108950C948B0D9091520292FD10C0FC
:101BE00098E0899F90011124262B209379010E946F
:101BF0009A08809179018595859585950C94EA0DD3
:101C00000C949A081092790180E00C94EA0D2091CE
:101C100079018095822380937901982F977099F4A8
:101C200030E0482F082E000C550B2417350759F0CB
:101C30009091520292FD07C08595859585950E94E9
:101C4000BB080C94020E08959091520292FB222739
:101C500020F9281769F080FB92F990935202809145
:101C60005102909152020E94720E82E00C94070E73
:101C700008958091520282FB882780F991E089279C
:101C80000C94240E81E00C94240E80E00C94240E1D
:101C90006FEF7FEF80E090E00C947D1D80E090E09E
:101CA0000E945A1D21E0893E9E4F09F020E0822FBC
:101CB000089582E090E00C94521D83E090E00C9433
:101CC000521DCF9384E090E00E94521DC82F82E203
:101CD00090E00E94521D2C2F30E0A901582BCA0120
:101CE000CF910895CF93C92F682F84E090E00E9490
:101CF000601D6C2F82E290E0CF910C94601DAB01CF
:101D0000BC018FE090E00C94711DAB01BC0183E13C
:101D100090E00C94711D60E070E0CB010C94850E96
:101D200060E070E0CB010E947F0E0C948B0E69EE98
:101D30007EEF80E090E00E947D1D60E082E090E018
:101D40000E94601D60E083E090E00E94601D1092A0
:101D5000350110923601109237011092380160E07F
:101D600084E090E00E94601D60E082E290E00E94CA
:101D7000601D60E085E090E00E94601D60E086E00C
:101D800090E00E94601D6FEF87E090E00E94601D70
:101D900040E050E0BA0188E090E00E94711D60E0F0
:101DA0008DE090E00E94601D40E050E0BA0188E1C3
:101DB00090E00E94711D60E087E190E00E94601D4C
:101DC00040E050E0BA018CE190E00E94711D60E0BB
:101DD00070E080E290E00E947D1D40E050E0BA019A
:101DE00088E190E00E94711D0C94900E0C94970E67
:101DF000682F8EE090E00C94601D0E94BF196093E4
:101E00009701709398018093990190939A01609340
:101E10009301709394018093950190939601089596
:101E20000E94BF1960939701709398018093990164
:101E300090939A0160938F01709390018093910128
:101E400090939201089584B7806884BF84B78068B6
:101E500084BF089581E008950C942A0F08950C948E
:101E60002E0F0C942E0F0C94310F0C942E0F0C94FB
:101E7000350F0C942E0F0E94230F8EEF91E10E94DC
:101E8000D9180E94390F0C94370F0E942F0F0C9411
:101E90002E0F0E9418120C94A7030E94AC190E94E6
:101EA000FD120E94490F0E9485170C94330F5F9218
:101EB0006F927F928F929F92AF92BF92CF92DF925A
:101EC000EF92FF920F931F93CF93DF93CDB7DEB7BF
:101ED0002A970FB6F894DEBF0FBECDBF0E94121333
:101EE000C82E81110E94FD0E35E8832E31E0932E1D
:101EF00000E010E0502E802F0E943C125C01F401A3
:101F0000619071904F016826792661147104B1F4D3
:101F10000F5F1F4F0530110569F78FEF89838A83A3
:101F20001B820E94B3198160782F9D838C83498125
:101F30005A816B818D810E94C3033AC080919B01BD
:101F400081FD0E944512D12CEE24E394F12CC301B3
:101F50008E219F21892B29F10E942C0F8823A9F023
:101F6000DE825F82AE20BF2081E0AB2809F480E0F2
:101F700088870E94B3198160782F9A8789874E815C
:101F80005F8168858A850E94C303000F111FF801D5
:101F9000EB57FE4F80819181E826F926F182E0829D
:101FA00007C0D394EE0CFF1CFEE0DF12D0CFB0CF01
:101FB00081E0C11001C080E02A960FB6F894DEBF20
:101FC0000FBECDBFDF91CF911F910F91FF90EF908A
:101FD000DF90CF90BF90AF909F908F907F906F9049
:101FE0005F9008950E94570F0E94971781110E94D9
:101FF000100F0E9413150C94B803CF93DF930E9427
:102000002711EC01811521E5920708F045C08115E3
:1020100030E5930708F094C0883E910528F5803E8E
:10202000910508F0F8C0883A910570F4853A910559
:1020300008F07CC08130910509F475C008F4E8C04F
:10204000049708F0E8C0E4C08F3B910508F0E0C0B9
:10205000C85AD0E0CC0FDD1FC555DF4F0990D8819D
:10206000C02DCE019464D8C0811540E2940758F485
:10207000811551E0950708F0CEC08D3E910508F41A
:10208000C7C09065C9C0C11580E4D80708F4C0C0B6
:10209000DF70CE01906AC0C0811525E59207A8F4D3
:1020A000811534E5930708F095C0811543E5940741
:1020B00008F07BC0811552E5950708F061C0D82F64
:1020C000CC27CE01816F906AA7C0C11589E5D807DA
:1020D000A0F4C11528E5D20708F082C0C11536E585
:1020E000D30708F095C08C2F0E94BB118F7190E030
:1020F000D82FCC27CE0190628FC0C1154AE5D407F6
:1021000008F474C0CE0190568115904208F080C04A
:102110008D2F8F710E94BB11DD27D0628F71AE01B0
:10212000582BCA0179C081E090E076C0C55AD0E052
:10213000C752DF4F8881C82FD0E0CE0190646CC0B9
:1021400074E0969587957A95E1F7282F23703C2FB8
:10215000337081E090E002C0880F991F3A95E2F752
:102160009C68AC01522B9A019C2F9F709695969576
:1021700050E2959FE0011124C9018C2B9D2B4CC08E
:102180008370992721E030E002C0220F331F8A9527
:10219000E2F79C2F9695969580E2989FE001112496
:1021A000C22BD32BCE019C6837C08370992721E0C6
:1021B00030E002C0220F331F8A95E2F79C2F9695DC
:1021C000969540E2949FE0011124C22BD32BCE01BF
:1021D0009A6822C0D82FCC27CE01846F906A1CC089
:1021E000DC2FCC27CE01806F906A16C08C2F8F70A9
:1021F0000E94BB1194E0D695C7959A95E1F7CF70F0
:10220000D0E0DC2FCC27D0699E01282BC90104C067
:1022100080E090E001C0CE01DF91CF91089526E4E7
:10222000829FC0011124FC012EE0729FE00DF11D80
:102230001124E60FF11DEE0FFF1FE459FF4F8591AA
:10224000949108950E940F110E94FD0F0895823805
:10225000910569F1B0F48133910509F46DC048F43A
:102260008932910509F463C08A32910509F469C085
:1022700008958533910509F455C089339105B9F066
:102280000895833E910569F138F4803E9105B1F0DF
:10229000823E910509F10895863E9105A9F1873E98
:1022A0009105B9F1843E910509F064C023C02091E5
:1022B000510220FD4FC021FD4DC008958091510273
:1022C00080FD44C08091520280FF44C08091510241
:1022D00084FD42C083EE4DC08091510282FF38C020
:1022E000F5CF8091510282FD33C08091520280FD72
:1022F00031C0ECCF8091520281FF32C080915102F7
:1023000084FD2AC087EE35C08091510283FF26C02C
:10231000F5CF8091510283FD21C08091520281FD51
:102320001FC0ECCF8091510285FD1CC01DC0809163
:10233000510285FD19C016C08091510286FD16C05C
:1023400017C08091510286FD13C010C089E311C0EF
:1023500082EE0FC080EE0DC080E00BC086EE09C09B
:1023600084EE07C089E205C085E303C08AE201C0AC
:1023700081E390E008959091510292FF0DC0282FC3
:102380002871283019F4877F846006C0282F2471B3
:10239000243011F48B7F886093FF0DC0282F2871A3
:1023A000283119F4877E846106C0282F24712431D6
:1023B00011F48B7E88612091520220FF0DC0382FCE
:1023C0003871383019F4877F816006C0382F317139
:1023D000313011F48E7F886021FF0DC0282F2871C5
:1023E000283119F4877E816106C0282F217121319F
:1023F00011F48E7E886194FD877E089580E00895B3
:102400000C94480E0E9412138FE39CE90197F1F798
:1024100000C000000E94121380E00E943C1280FF66
:1024200004C00E9400120C94001A08950C94021229
:102430000E944E0E811102C00E94F60E0E94590E9B
:1024400080939B010E94610E9093520280935102EF
:102450000E9416120E945D0E682F70E080E090E0EE
:102460000E943A08609131017091320180913301EC
:10247000909134010C947208E82FF0E0EE0FFF1FEA
:10248000E35AFD4F808191810895089580EA8A95ED
:10249000F1F7089500C008950C94461208950C9425
:1024A0004E120C944F120C944E120C945312F8943A
:1024B000E82FE295EF70F0E031A9282F2F7081E02E
:1024C00090E001C0880F2A95EAF7982F9095932302
:1024D00091AB92A9892B82AB789408950F931F93A7
:1024E000CF93DF93CAEED0E089918F3F11F00E9425
:1024F000571280E0CF3ED807B9F7CCEDD0E00AEE16
:1025000010E089918F3F11F00E9457120C171D07A0
:10251000C1F7DF91CF911F910F910895BF92CF9294
:10252000DF92EF92FF920F931F93CF93DF938C0173
:10253000C62FD0E0CE0186519F4F6C01FC019081E7
:102540009F3F09F450C0B62EF894E92FE295EF7042
:10255000F0E081A99F7021E030E001C0220F9A9540
:10256000EAF7822B81AB82A92095282322AB7894AD
:102570000E944A12ECEDF0E04AEE50E021E030E03B
:10258000E12CF12C61916F3F89F0A62FA295AF70DD
:10259000B0E0D0968C9190E06F7002C095958795D1
:1025A0006A95E2F780FD02C0C90102C080E090E0B8
:1025B000E82AF92A220F331F4E175F0719F7F60191
:1025C00080818F3F11F00E94571261E0E114F10405
:1025D00009F460E08B2D0E944C12CC0FDD1FC00F60
:1025E000D11FF982E882DF91CF911F910F91FF9067
:1025F000EF90DF90CF90BF9008950E946E128AE016
:10260000EDE5F2E0DF01982F1D929A95E9F7E3E5F9
:10261000F2E0DF011D928A95E9F785E00E945D13E3
:102620000C943203FF920F931F93CF93DF93CDB798
:10263000DEB72A970FB6F894DEBF0FBECDBF8E016E
:102640000F5F1F4F8AE0F80111928A95E9F7F12C8C
:102650006F2DC8010E948E12F394F5E0FF12F8CF9F
:102660004AE050E0B80183E592E00E94451DFF2456
:10267000F394009709F4F12C892B41F08AE0F801DA
:10268000A3E5B2E001900D928A95E1F72F2D45E088
:102690006DE572E083E592E00E945E130E943403D0
:1026A0008F2D2A960FB6F894DEBF0FBECDBFDF91F7
:1026B000CF911F910F91FF9008950895FF920F936E
:1026C0001F93CF93DF93F82E092F162FD72FC42FE8
:1026D000222349F081E080939E010E94B3199093D8
:1026E0009D0180939C0180919E018823D9F0809167
:1026F0009C0190919D010E94CB19059798F0EF2DB8
:10270000F02FA12FBD2F80E090E04C2F50E08417D8
:10271000950734F4219131912D933D930196F7CF94
:1027200010929E01DF91CF911F910F91FF9008951C
:102730000E941A1A0E944D0F0C942B1A0E94A11984
:102740000E94131A0E943B0F0E9498130E94391A8C
:102750000E94450FFBCF8091A50180FF06C06091CC
:10276000690070E0660F771F26C081FF04C060918A
:10277000690084E005C082FF07C06091690088E0BD
:10278000689FB001112417C09091A4019923D1F042
:1027900060916800961788F72091690088E0289F6B
:1027A00090011124929FA001939F500D112470E07D
:1027B000CA010E94171D6038710540F4611571054A
:1027C00019F406C068E070E0862F08958FE7089539
:1027D00081E008958091A50180FF08C060916500A7
:1027E00070E0759567957595679521C081FF06C066
:1027F0006091650070E07595679519C082FF04C00F
:102800006091650070E010C09091A301992399F048
:10281000609164009617A0F780916500899FC001C0
:10282000112470E00E94171D6038710540F4611595
:10283000710519F406C061E070E0862F08958FE7F6
:10284000089581E008958D3E21F40E94AB13819597
:1028500004C08E3E29F40E94AB138093A901089511
:102860008F3E21F40E94AB13819504C0803F29F470
:102870000E94AB138093A8010895893F19F40E9428
:10288000EA1305C08A3F31F40E94EA1381958093D0
:10289000AA0108958B3F21F40E94EA13819504C098
:1028A0008C3F29F40E94EA138093AB0108959FE0C6
:1028B000980F983078F421E030E0A90102C0440F6D
:1028C000551F9A95E2F7CA019091A701892B809331
:1028D000A70108958D3F21F48091A50181600BC06F
:1028E0008E3F21F48091A501826005C08F3F29F4BD
:1028F0008091A50184608093A50108958D3E39F4EF
:102900009091A90197FF35C01092A90159C08E3E40
:1029100029F49091A9011916BCF32BC09091A8013C
:102920008F3E29F497FF25C01092A80149C0803F2F
:1029300019F41916CCF31DC09091AA01893F29F40E
:102940001916BCF41092AA013BC08A3F19F497FFF4
:1029500010C0F8CF8B3F39F49091AB0197FF09C0BD
:102960001092AB012DC08C3F21F49091AB01191650
:10297000BCF39FE0980F983080F421E030E0A9018B
:1029800002C0440F551F9A95E2F7CA0180959091B5
:10299000A70189238093A70113C08D3F21F4809163
:1029A000A5018E7F0BC08E3F21F48091A5018D7F04
:1029B00005C08F3F29F48091A5018B7F8093A501ED
:1029C0008091A801811106C08091A901811102C0E6
:1029D0001092A4018091AA01811106C08091AB01DF
:1029E000811102C01092A30108950E94B319209191
:1029F000A801211104C02091A901222321F0909364
:102A0000A2018093A1012091AA01211104C020916B
:102A1000AB01222321F09093A00180939F0186EACD
:102A200091E00C94FA18EF92FF920F931F93CF93BB
:102A3000DF9300D000D000D0CDB7DEB786E0E6EA65
:102A4000F1E0DE01119601900D928A95E1F7E09098
:102A5000A801F090A9010091AA011091AB01109278
:102A6000A8011092A9011092AA011092AB01E110E5
:102A700003C0FF2009F45DC08091A1019091A201E3
:102A80000E94CB19AC019091A401992339F02091B7
:102A90006A0030E02417350758F04BC020916B00D6
:102AA0008AE0289F900111242417350718F041C0AF
:102AB0009F3F19F09F5F9093A401EE2061F00E9468
:102AC000AB131E1414F09FEF01C091E0989F902D5E
:102AD00011249093A801FF2061F00E94AB131F14F2
:102AE00014F09FEF01C091E0989F902D11249093D6
:102AF000A9013091A8013323E1F02091A9012223FB
:102B0000C1F045EB3403C0011124992319F09093CF
:102B1000A80103C081E08093A80135EB2303C00125
:102B20001124992319F09093A90103C081E08093A7
:102B3000A901011103C0112309F45DC080919F0117
:102B40009091A0010E94CB19AC019091A30199230F
:102B500039F02091660030E02417350758F04BC05B
:102B6000209167008AE0289F9001112424173507DF
:102B700018F041C09F3F19F09F5F9093A30100237D
:102B800061F00E94EA13101614F09FEF01C091E06B
:102B9000989F902D11249093AA01112361F00E9417
:102BA000EA13111614F09FEF01C091E0989F902D49
:102BB00011249093AB013091AA013323E1F02091CD
:102BC000AB012223C1F045EB3403C001112499234A
:102BD00019F09093AA0103C081E08093AA0135EB1C
:102BE0002303C0011124992319F09093AB0103C072
:102BF00081E08093AB018091A80181110BC080918D
:102C0000A901811107C08091AA01811103C080919F
:102C1000AB0181110E94F514EB82FC820D831E83AF
:102C200086E0FE013196A6EAB1E001900D928A9508
:102C3000E1F726960FB6F894DEBF0FBECDBFDF9149
:102C4000CF911F910F91FF90EF900895E6EAF1E088
:102C500086E0DF011D928A95E9F71092A401109297
:102C6000A3011092A5010895CF93DF93EC01FB011E
:102C70008281882309F43CC1C430FDE5DF0760F49C
:102C8000CB3F9CE5D90788F49E0122503C45243176
:102C9000310508F02EC109C0C236EDE5DE0729F086
:102CA000C63AFDE5DF0709F024C10E94610E90934A
:102CB000520280935102C1318CE5D80709F4C6C095
:102CC00008F042C0C930ECE5DE0709F49BC000F50E
:102CD000C5308CE5D80709F485C078F4C330ECE53D
:102CE000DE0709F478C008F07AC0C230DC4509F08C
:102CF000F5C0809151028160EFC0C7309CE5D907D3
:102D000009F478C008F07AC0809151028061E4C073
:102D1000CD30FCE5DF0709F487C058F4CB309CE5E3
:102D2000D90709F479C008F07BC08091510288600E
:102D30006FC0CF30FCE5DF0709F480C008F082C027
:102D400080915102877FC8C0CE3F9CE5D90709F426
:102D500071C000F5C531FCE5DF0709F485C068F4F2
:102D6000C3319CE5D90709F475C008F095C00E94ED
:102D7000E207809151028F77AFC0CC3FFCE5DF07BF
:102D8000A9F108F054C0CB3FDC4509F0A7C0809101
:102D9000520240C0C230EDE5DE0709F489C058F4A4
:102DA000C1158DE5D80709F45AC008F069C08091B3
:102DB000520282602FC0C236EDE5DE0709F47CC006
:102DC000C63AFDE5DF0709F481C0C330DD4509F0EF
:102DD00085C080E06EC08091510282607DC080918C
:102DE000510216C080915102886076C080915202D3
:102DF00082604FC08091510280626EC0809151020A
:102E000080646AC00E94E20780915102806864C0B9
:102E1000846062C081603DC0809151028E7F5CC041
:102E2000809151028D7F58C08091510216C08091CF
:102E3000520218C0809152028D7F2BC080915102A6
:102E40008F7E4AC0809151028F7D46C08091510291
:102E50008F7B42C080915102877F8B7F3DC08091E4
:102E600052028D7F8E7F15C08091510282FB2227F6
:102E700020F991E0922790FB82F990FB83F92CC016
:102E800080915202982F909591708E7F892B90FBA4
:102E900081F98093520222C00E94E2078091510280
:102EA00087FB222720F991E0922790FB87F914C035
:102EB00081E00E94F80E12C08091510284FB22270B
:102EC00020F991E0922790FB84F906C0809151028D
:102ED000982F909590FB80F9809351028091510238
:102EE000909152020E94720E0E94E20780E001C09F
:102EF00081E0DF91CF9108958FE891E00197F1F79C
:102F000000C0000008950C94D702D098D89AD198A8
:102F1000D99A0E947C1789B3982F9170C99902C0E1
:102F200080E001C082E0892B8093AE010895E0919A
:102F3000AE01EE0FEE0FE093AE0149B3842F817026
:102F400090E049B341FB222720F930E041FF02C065
:102F500022E030E0822B932B8E2B8093AE018F707A
:102F6000E82FF0E0E151FF4F90818091AD01890F92
:102F70008093AD0184305CF08091AC018F5F8093D1
:102F8000AC0160E080E00E94831721E001C020E0F6
:102F90008091AD018D3F54F48091AC0181508093BC
:102FA000AC0161E080E00E94831721E08091AD01D7
:102FB000082E000C990B64E070E00E94171D8093AE
:102FC000AD01822F0895CF93DF9386319C4541F563
:102FD000EB010E94650D982F8A812091620030914B
:102FE0006300882379F09A7A81E009F480E0809385
:102FF000AF01911102C069E201C065E3C9010E94FD
:1030000076190AC08091AF01811102C069E201C046
:1030100065E3C9010E9478190E94A70D80E001C0F4
:1030200081E0DF91CF9108950F931F93CF93DF93AA
:10303000C42FD22FFC0182818823C9F04093B201B2
:103040000E94B3199093B1018093B00180E28C0F7C
:10305000883008F057C0C77081E001C0880FCA955A
:10306000EAF7DF91CF911F910F910C944505809164
:10307000B201481330C08091B0019091B1010E941B
:10308000CB19883C910538F510E21D0FCD17B9F02A
:1030900080E28C0F883040F4C77081E001C0880F57
:1030A000CA95EAF70E944C05183028F581E09D2F5B
:1030B000977001C0880F9A95EAF70E944505802F06
:1030C0000E943C051830F0F4D77081E001C0880FF1
:1030D000DA95EAF70AC080E28C0F883098F4C7705E
:1030E00081E001C0880FCA95EAF7DF91CF911F9167
:1030F0000F910C944C05802FDF91CF911F910F9170
:103100000C943C05DF91CF911F910F9108950F937F
:103110009C01CB01243F4CE5340731F188F4293D73
:10312000FCE53F07D9F02A3D4CE5340779F1283D0D
:103130003C45A9F506E221EE41EE68ED7CE52BC0A9
:10314000263FFCE53F07E1F0A8F0273F3C4539F575
:1031500007E225EE46EE67EF7CE51DC007E225EEAF
:1031600045EE69ED7CE517C006E221EE40EE64EF26
:103170007CE511C007E225EE44EE65EF7CE50BC06F
:1031800006E221EE42EE66EF7CE505C008E221E0B2
:1031900045EE6AED7CE50E94141880E008C0FC0151
:1031A0008281882319F01092B20101C081E00F9151
:1031B0000895909301018093000108959093B801C0
:1031C0008093B7010895E091B701F091B80130976D
:1031D00021F00190F081E02D099480E00895E091C4
:1031E000B701F091B801309721F00280F381E02D12
:1031F00009940895E091B701F091B801309739F042
:1032000022E0DC012C930480F581E02D09940895DF
:103210002091B5013091B6012817390771F09093CC
:10322000B6018093B501E091B701F091B8013097F4
:1032300021F00680F781E02D099408952091B301D3
:103240003091B4012817390771F09093B40180933D
:10325000B301E091B701F091B801309721F00084FB
:10326000F185E02D09940895FC01329697E080E005
:10327000915029F021912223D9F38F5FF9CF08953E
:10328000662349F0FC01329608962191621729F0D5
:10329000E817F907D1F780E0089581E008959C01CF
:1032A000FC0132969FEF80E04191461789F09F3FE5
:1032B00019F4411101C0982F8F5F8630A9F79F3F05
:1032C00039F0F901E90FF11D97FDFA956283089530
:1032D00008959C012A5F3F4FFC014281461301C0C3
:1032E0001282019682179307B9F708950C944F192B
:1032F0000C946919029626E0FC0111922A95E9F7CF
:10330000089508950C9481190C9482190C948119D4
:103310000C9481190C948119CF930E9488190E94F2
:1033200012130E948619C0E08C2F0E943C12892B38
:1033300029F4CF5FC530C1F780E001C081E0CF91B3
:10334000089508958091BB0181110C94980308950C
:103350000E94E2070C949C038BE083BF8AEF8CBF32
:1033600082E089BF08952FB7F89480916702909109
:103370006802A0916902B0916A022FBF08952FB729
:10338000F89460916702709168028091690290914F
:103390006A022FBF08959C014FB7F894809167028D
:1033A00090916802A0916902B0916A024FBF821B9E
:1033B000930B089578941F920F920FB60F921124D9
:1033C0008F939F93AF93BF93809167029091680210
:1033D000A0916902B0916A020196A11DB11D80936E
:1033E000670290936802A0936902B0936A02BF914A
:1033F000AF919F918F910F900FBE0F901F901895D6
:1034000098E088E10FB6F894A89581BD0FBE91BDF4
:10341000A895F894D8E0CEE528E3299320E02993F5
:1034200014BEFFCF08950E94B3199093BA01809300
:10343000B90108950E94FC1C8B9A80E0815041F0F4
:10344000A895EFE9FFE03197F1F700C00000F6CF53
:103450008B98789408950E941F1B0E94DE182FEF0E
:1034600080E792E0215080409040E1F700C00000EA
:10347000089580919202882389F0109292020E940E
:10348000B3199093BA018093B9018091BB0188234D
:10349000D1F11092BB010E94A81911C08091BB010B
:1034A000811111C08091B9019091BA010E94CB198C
:1034B000069728F081E08093BB010E94A2198091B9
:1034C000BB01882301F10E94A2190E948C19882354
:1034D00039F1F89421B3939A822F8C6081BB92B317
:1034E0008CE0982792BB3FE748E391E031504040A1
:1034F0009040E1F700C0000092B3892782BB21BB56
:103500009398789408950E94051C809198028823CE
:1035100029F08091760284FD0E94F20F0C94C61A65
:10352000089580915002089508959091C1019813D3
:1035300007C02091BF013091C00126173707A9F0BD
:103540008093C1017093C0016093BF018093BC015F
:103550007093BE016093BD018091AF0284FF05C0EE
:1035600063E08CEB91E00C94011C0895BC0184E0B5
:103570000C94951ABC0183E00C94951A2091AF022B
:1035800024FF03C066E00C94011C0895CF93DF93E1
:10359000CAE0D0E08091760284FF18C08091CD010E
:1035A0009091CE019817E1F028E0829FC00111248C
:1035B00068E081539E4F0E94FD1B8091CD0190E0F9
:1035C00001968F7099278093CD010AC00E94051C37
:1035D0008FE99FE00197F1F700C000002197D1F635
:1035E000DF91CF910895CF93DF93EC01A091CE01AD
:1035F000B0E0CD0101968F7099272091CD01281759
:1036000079F093E0AA0FBB1F9A95E1F7A153BE4F43
:1036100098E0FE0101900D929A95E1F78093CE011A
:103620000E94051C0E94C61A88E0FE01A5ECB1E0CC
:1036300001900D928A95E1F7DF91CF9108958CE684
:1036400090E00895FC01808180768032A1F581812F
:10365000813061F484819581892B69F585EC91E055
:10366000909394028093930288E00895823041F40D
:103670008FE492E0909394028093930281E0089506
:103680008A3021F4838180934F0215C0893099F4E8
:10369000828193818115924081F484819581892B67
:1036A00061F481E08093C401868197819093C30186
:1036B0008093C20102C080E008958FEF08952091A9
:1036C000C2013091C301232B71F02091C40121303C
:1036D00051F4FC018081809350021092C30110923A
:1036E000C20181E008958FEF08950895FC01938150
:1036F0009330D9F068F4913081F0923009F059C0DC
:1037000084E891E090939402809393028BE3089570
:10371000913249F19232B9F14CC08FEB91E0909324
:1037200094028093930282E108958281813099F01E
:1037300050F08230F1F581ED91E090939402809306
:10374000930280E108958DEF91E09093940280932D
:10375000930284E0089583EE91E090939402809325
:10376000930288E108958281882329F0813009F548
:103770008FEA91E002C086E991E0909394028093F1
:10378000930289E0089584819581009751F0019713
:1037900081F481E092E090939402809393028BE70E
:1037A00008958CE792E0909394028093930280E4D2
:1037B000089580E008951F93CF93DF93162FEA01B9
:1037C000288124FF05C0398128E82327298302C0E6
:1037D0002AE52883212FFC01CE010296DC013191DC
:1037E0003D9321501216DCF3612F0E9492011C5F61
:1037F0001883DF91CF911F91089546E752E00C9412
:10380000DB1B4FEA52E00C94DB1BCF93DF936091FC
:103810009502635067FD93C080919102CCE0D0E0A7
:10382000C81BD109C756DD4F80919002803120F42A
:10383000CE010E94751B81C08D3209F06EC06830C8
:1038400009F07BC083EC80936B028AE5809379005A
:1038500010928F028881807621F0CE010E94221B77
:1038600049C09A81109274028981811106C0109218
:10387000750224E732E082E038C0853019F4909375
:10388000960230C08630A1F48B81813041F08230C5
:1038900031F0833021F0813211F0823221F4CE01F7
:1038A0000E94761B01C080E090E490938F0222C0BA
:1038B000883089F0893019F49093980213C08A30C7
:1038C00069F08B3079F48BE4809377028093B002B7
:1038D0008093830207C028E932E002C024E732E087
:1038E00081E003C024E732E080E03093940220932B
:1038F000930209C08F3F39F4988197FD8E8190E83B
:1039000090938F0207C09F81911104C09E819817E8
:1039100008F4892F8093780010C080918F0287FF70
:103920000CC0CE010E945F1B8F3F21F48EE180937B
:10393000790003C081111092780010929502809155
:10394000790084FF4CC0809178008F3F09F447C014
:10395000C82F893008F0C8E08C1B809378009091C4
:103960006B0288E8892780936B02CC2359F1809100
:1039700093029091940220918F0226FF12C0ABE631
:10398000B2E02C2FAC014B565240FA01EA0FFB1F5C
:10399000E4911196EC931197215011962111F5CFD6
:1039A00008C0ECE6F2E0DC012C2F3D913193215070
:1039B000E1F701962FEF2C0F820F911D9093940247
:1039C000809393026C2F8CE692E00E949201CC5F70
:1039D000CC3019F08FEF80937800C093790084E1A8
:1039E00090B39C7031F48150D9F7109296021092E6
:1039F0008E02DF91CF910895CF93DF9385B78860D2
:103A000085BF8BB780688BBFC6E7D2E08BE4898324
:103A1000AFEAB2E011968C931197E2E8F2E081836D
:103A20008AE588838C938083DF91CF91089597FBFB
:103A3000072E16F4009407D077FD09D00E94311D9F
:103A400007FC05D03EF4909581959F4F08957095A1
:103A500061957F4F0895EE0FFF1F0590F491E02DC3
:103A60000994AA1BBB1B51E107C0AA1FBB1FA617C5
:103A7000B70710F0A61BB70B881F991F5A95A9F717
:103A800080959095BC01CD010895FB01DC0104C037
:103A90008D910190801921F441505040C8F7881B46
:103AA000990B0895E199FECF9FBB8EBBE09A9927B1
:103AB0008DB30895A8E1B0E042E050E00C94851D7C
:103AC000262FE199FECF9FBB8EBBE09A01970DB2E6
:103AD000021631F02DBB0FB6F894E29AE19A0FBEB0
:103AE00008950396272F0E94611D0E94601D252FB7
:103AF0000E94611D242F0C94611D0196272F0E94A6
:103B0000611D0C94601DDC01CB01FC01E199FECF2D
:103B100006C0FFBBEEBBE09A31960DB20D9241504C
:0A3B20005040B8F70895F894FFCF65
:103B2A00C8007B01280850011E0A1401911AF31AD1
:103B3A00BE1ABA1AB61A941AFF5AE200E900EA0043
:103B4A00B500B600B700CD008301CC008A0192010E
:103B5A0094012102230224022502260227022A02B4
:103B6A00B300B4006F007000818283E200E900EACA
:103B7A0000B500B600B700CD008301CC008A0192DF
:103B8A000194012102230224022502260227022A85
:103B9A0002B300B4006F0070008182839596973754
:103BAA003635343332319493926405063007FF0078
:103BBA00FF0100010000FFFF0000010001FF0000FB
:00000001FF
